:020000040800F2
:1000000000060020E1020008E3020008E302000805
:10001000E3020008E3020008E3020008E30200082C
:10002000E3020008E3020008E30200081D320008B2
:10003000E3020008E3020008E3020008E30200080C
:10004000E3020008E3020008E3020008E3020008FC
:10005000E3020008E3020008E3020008E3020008EC
:10006000E3020008E3020008E3020008BD110008F3
:10007000E5110008111200083D120008691200087D
:1000800091120008BD120008E3020008E302000814
:10009000E3020008E3020008E3020008E3020008AC
:1000A000E3020008E3020008E3020008E30200089C
:1000B000E3020008E3020008E3020008E30200088C
:1000C000E3020008E3020008E3020008E30200087C
:1000D000E3020008E3020008E3020008014A000806
:1000E000E3020008E3020008E3020008E30200085C
:1000F000E3020008E3020008E3020008E912000836
:10010000E3020008E30200083D4A0008E302000899
:10011000E3020008154A0008E3020008E3020008B1
:10012000151300083D130008691300089513000813
:10013000C1130008E3020008E3020008E30200081C
:10014000E3020008E3020008E3020008E3020008FB
:10015000E91300081514000841140008E302000820
:10016000E3020008E3020008E3020008E3020008DB
:10017000E3020008093E0008E3020008E302000869
:10018000E3020008E3020008294A0008E30200082D
:10019000E3020008E3020008E3020008E3020008AB
:1001A000E3020008E3020008E3020008E30200089B
:1001B000E3020008E3020008E3020008E30200088B
:1001C000E3020008E3020008E3020008E30200087B
:1001D000E3020008F53D0008E3020008E30200081E
:1001E000E3020008E3020008E3020008E30200085B
:1001F000E3020008E3020008E3020008E30200084B
:10020000E3020008E3020008E3020008E30200083A
:10021000E3020008E3020008E3020008E30200082A
:10022000E3020008E3020008E3020008E30200081A
:10023000E3020008E3020008E3020008E30200080A
:10024000E3020008E3020008E3020008E3020008FA
:10025000E3020008E3020008E3020008E3020008EA
:10026000E3020008E3020008E3020008E3020008DA
:10027000E3020008E3020008E3020008E3020008CA
:10028000E3020008E3020008E3020008E3020008BA
:10029000E3020008E3020008E3020008E3020008AA
:1002A000E3020008E3020008E3020008E30200089A
:1002B000E3020008E3020008E3020008E30200088A
:1002C000E3020008E3020008E3020008E30200087A
:1002D000E3020008E3020008E3020008E30200086A
:1002E00002E000F000F8FEE772B6374880F30888B5
:1002F000364880F3098836483649086040F20000E5
:10030000CCF200004EF63471CEF200010860BFF36B
:100310004F8FBFF36F8F40F20000C0F2F0004EF637
:100320008851CEF200010860BFF34F8FBFF36F8F8B
:100330004FF00000E1EE100A4EF63C71CEF20001E3
:100340000860062080F31488BFF36F8F02F0C8FFA7
:1003500004F010F94FF055301F491B4A91423CBF41
:1003600041F8040BFAE71D49184A91423CBF41F895
:10037000040BFAE71A491B4A1B4B9A423EBF51F83D
:10038000040B42F8040BF8E700201849184A914280
:100390003CBF41F8040BFAE702F0E0FF04F06EF90D
:1003A000144C154DAC4203DA54F8041B8847F9E7A6
:1003B00000F042F8114C124DAC4203DA54F8041B21
:1003C0008847F9E702F0C8BF00060020002200209D
:1003D0000000000808ED00E00000002000060020FA
:1003E000884F0008002200206C220020702200208C
:1003F0006C510020E0020008E0020008E002000862
:10040000E00200082DE9F04F2DED108AC1F80CD064
:10041000D0F80CD0BDEC108ABDE8F08F002383F338
:1004200011882846A047002002F0B0F9FEE702F04C
:100430003BF900DFFEE7000038B500F04DFC00F0AE
:100440000FFE02F0ABFE054602F0DEFE0446C0B928
:100450000E4B9D4217D001339D4241F2883512BFA9
:10046000044600250124002002F0A2FE0CB100F099
:1004700073F800F095FD284600F01CF900F06CF8C8
:10048000F9E70025EFE70546EDE700BF010007B0FB
:1004900008B500F0EDFBA0F120035842584108BD1B
:1004A00007B5042101900DEB010000F0FFFB03B044
:1004B0005DF804FB38B5302383F3118817480368CF
:1004C0000BB102F02FFA0023154A4FF47A7113484A
:1004D00002F01EFA002383F31188124C236813B133
:1004E0002368013B2360636813B16368013B636069
:1004F0000D4D2B7833B963687BB9022000F0B2FC54
:10050000322363602B78032B07D163682BB9022059
:1005100000F0A8FC4FF47A73636038BD70220020AD
:10052000B50400089023002088220020084B187092
:1005300003280CD8DFE800F008050208022000F0CC
:1005400083BC022000F070BC024B00225A6070474E
:100550008822002090230020F8B5504B504A1C46BA
:100560001968013100F0998004339342F8D1626830
:100570004C4B9A4240F291804B4B9B6803F10063D5
:1005800003F500339A4280F08880002000F0BEFB23
:100590000220FFF7CBFF454B0021D3F8E820C3F83A
:1005A000E810D3F81021C3F81011D3F81021D3F8B4
:1005B000EC20C3F8EC10D3F81421C3F81411D3F8CD
:1005C0001421D3F8F020C3F8F010D3F81821C3F8A1
:1005D0001811D3F81821D3F8802042F00062C3F834
:1005E0008020D3F8802022F00062C3F88020D3F866
:1005F0008020D3F8802042F00072C3F88020D3F826
:10060000802022F00072C3F88020D3F8803072B6C8
:100610004FF0E023C3F8084DD4E90004BFF34F8F37
:10062000BFF36F8F224AC2F88410BFF34F8F536914
:1006300023F480335361BFF34F8FD2F8803043F6F9
:10064000E076C3F3C905C3F34E335B0103EA060C3E
:1006500029464CEA81770139C2F87472F9D2203BFD
:1006600013F1200FF2D1BFF34F8FBFF36F8FBFF3A2
:100670004F8FBFF36F8F536923F40033536100230F
:10068000C2F85032BFF34F8FBFF36F8F302383F325
:100690001188854680F308882047F8BD00000208CD
:1006A00020000208FFFF0108002200200044025839
:1006B00000ED00E02DE9F04F95B0DFF8D892202250
:1006C000FF21029004A8D9F8085000F013FCA84AB2
:1006D0001378A3B90121A74811700360302383F375
:1006E000118803680BB102F01DF90023A24A4FF4F0
:1006F0007A71A04802F00CF9002383F31188029B61
:1007000013B19E4B029A1A609D4A1378032B03D0B3
:1007100000231370994A53604FF0000B029C5E4611
:10072000DA46CDF804B0012000F08EFB24B1934BE3
:100730001B68002B00F02882002000F099FAB0F12D
:100740000008F3DB012000F06FFBA8F121031F2B51
:10075000E9D801A252F823F0D9070008F5070008EC
:100760008308000827070008270700082707000854
:100770000D090008FF0A0008F10900084D0A0008E9
:10078000730A0008990A000827070008AB0A000846
:10079000CF0A0008470B0008610800082707000877
:1007A0008F0B0008E507000861080008270700080C
:1007B0004D0A000827070008270700082707000838
:1007C0002707000827070008270700082707000851
:1007D00027070008830800080220FFF759FE0028B9
:1007E00040F0FF81029B02216648BBF1000F08BF69
:1007F0001C4640E04FF47A7000F03AFA071EF1DB35
:100800000220FFF745FE0028ECD0013F052F00F243
:10081000EA81DFE807F003070A0D10330520FFF730
:100820003FFE14E0D9F80000F9E7D9F80400F6E734
:10083000D9F80800F3E74FF01C08404608F1040817
:1008400000F066FAFFF72CFEB8F12C0FF5D101206D
:10085000019B4FF0000A00FA07F71F43FBB2019318
:1008600000F094FB2EB1019B03F00B030B2B08BF90
:1008700000240221444800F019FA54E7D9F80C008A
:10088000CDE7002EAED0019B03F00B030B2BA9D1BB
:100890000220FFF7FDFD07460028A3D00120002617
:1008A00000F034FA0220FFF741FE1FFA86FB58469B
:1008B00000F03CFA044688B1A8F1400258460136DF
:1008C0005142514100F042FA0028EED1BB460446A5
:1008D00002212E483E4600F0E9F924E72546012092
:1008E000FFF724FED9F80830AB4207D9284600F0BC
:1008F0000FFA013040F07A810435F3E70025204BF0
:10090000BB463E461D701D4B5D60A9E7002E3FF4BF
:1009100069AF019B03F00B030B2B7FF463AF022045
:10092000FFF704FE322000F0A3F9B0F10008FFF653
:1009300059AF18F003077FF455AF08EB0503D9F85A
:10094000082093423FF64EAFB8F5807F3FF74AAF9D
:100950000F4BB84503931FDD4FF47A7000F088F910
:100960000028FFF63FAF039B013703F8010BF0E7C8
:100970008C23002070220020B50400089023002062
:1009800088220020F04A0008E84A0008EC4A0008E3
:100990008C22002000220020C820FFF779FD0746A6
:1009A00000283FF41FAF1F2D11D8C5F1200204AB62
:1009B00025F003008F494245184428BF4246039260
:1009C00000F072FA039AFF218A4800F093FA4FEA86
:1009D000A803C8F3870287492846039300F092FAD8
:1009E000064600283FF474AF039B05EB830537E709
:1009F0000220FFF74DFD00283FF4F4AE00F0C4F9EB
:100A000000283FF4EFAE0027B846D9F80830BB42C3
:100A100018D91F2F11D8049B01330ED027F00303E0
:100A200014AA134453F8403C0C93404604220CA9EA
:100A3000043700F0ADFB8046E7E7384600F068F980
:100A40000C90F2E74046FFF72BFD09E700236421F5
:100A50000CA80C9300F020F900287FF4C3AE02200C
:100A6000FFF716FD00283FF4BDAE0C9800F082F9A8
:100A7000E9E7002364210CA80C9300F00DF900288D
:100A80007FF4B0AE0220FFF703FD00283FF4AAAECA
:100A90000C9800F071F9D6E70220FFF7F9FC002866
:100AA0003FF4A0AE00F080F9CDE70220FFF7F0FCA4
:100AB00000283FF497AE0CA9142000F07BF90390B6
:100AC000FFF7EEFC03990CA800F0F0F8C8E602204E
:100AD000FFF7DEFC00283FF485AE474B0CAF03F177
:100AE000100C1868083353F8041C3A46634503C2D7
:100AF0001746F6D11020FFF7D3FC1021E3E7322090
:100B000000F0B6F8071EFFF66DAEBB077FF46AAEC5
:100B100007EB0A03D9F8082093423FF663AE0220A0
:100B2000FFF7B6FC00283FF45DAE27F003075744FB
:100B3000BA453FF495AE50460AF1040A00F0E8F8D1
:100B4000FFF7AEFCF4E74FF47A70FFF7A1FC002842
:100B50003FF448AE00F018F9002849D0049B013357
:100B60000BD0082204A9002000F0CCF900283FD0C7
:100B70002022FF2104A800F0BDF92048022100F046
:100B800095F81F4801F008FE15B0BDE8F08F002E63
:100B90003FF428AE019B03F00B030B2B7FF422AE36
:100BA000002364210CA80C9300F076F80746002877
:100BB0007FF418AE0220FFF76BFC804600283FF45C
:100BC00011AE02210D4800F071F841F2883001F0B9
:100BD000E3FD0C9800F022FA46463C4600F0D6F9B8
:100BE000A1E506463CE64FF0000AFBE5BB466FE692
:100BF00037466DE68C220020D44A0008E84A0008F7
:100C0000A08601002DE9F84F4FF47A7306460D4691
:100C1000002402FB03F7DFF85080DFF8509098F9CA
:100C200000305FFA84FA5A1C01D0A34210D159F85F
:100C300024002A4631460368D3F820B03B46D84703
:100C4000854205D1074B012083F800A0BDE8F88F4D
:100C50000134042CE3D14FF4FA7001F09DFD002023
:100C6000F4E700BFDC230020102200201422002023
:100C7000002307B5024601210DF107008DF807306A
:100C8000FFF7C0FF20B19DF8070003B05DF804FB3B
:100C90004FF0FF30F9E700000A46042108B5FFF7DE
:100CA000B1FF80F00100C0B2404208BD074B0A46C8
:100CB00030B41978064B53F821400146236820468A
:100CC000DD69044BAC4630BC604700BFDC2300202C
:100CD00014220020A086010070B50A4E00240A4D9F
:100CE00002F074F8308028683388834208D902F013
:100CF00069F82B6804440133B4F5003F2B60F2D34C
:100D000070BD00BFDE2300209823002002F038B918
:100D100000F1006000F500300068704700F10060ED
:100D2000920000F5003002F0ADB80000054B1A68E3
:100D3000054B1B889B1A834202D9104402F042B82B
:100D40000020704798230020DE23002038B5044699
:100D5000074D29B128682044BDE8384002F04AB860
:100D60002868204402F034F80028F3D038BD00BFD2
:100D7000982300200020704700F1FF5000F58F10ED
:100D8000D0F8000870470000064991F8243033B1CC
:100D900000230822086A81F82430FFF7BFBF012032
:100DA000704700BF9C230020014B1868704700BFAC
:100DB0000010005C194B01380322084470B51D680F
:100DC000174BC5F30B042D0C1E88A6420BD15C6893
:100DD0000A46013C824213460FD214F9016F4EB10C
:100DE00002F8016BF6E7013A03F10803ECD1814206
:100DF0000B4602D22C2203F8012B0424094A168840
:100E0000AE4204D1984284BF967803F8016B013C4E
:100E100002F10402F3D1581A70BD00BF0010005C4B
:100E200024220020204B0008022804D1054B4FF457
:100E300000129A6170470128FCD1024B4FF4002246
:100E4000F7E700BF00100258022803D1044B20220C
:100E50009A6170470128FCD1014B0822F8E700BFD6
:100E600000100258022805D1064A536983F0200376
:100E7000536170470128FCD1024A536983F008038B
:100E8000F6E700BF0010025870B504464FF47A76BA
:100E90004CB1412C254628BF412506FB05F0641BBB
:100EA00001F07AFCF4E770BD002310B5934203D043
:100EB000CC5CC4540133F9E710BD0000013810B513
:100EC00010F9013F3BB191F900409C4203D11AB1A6
:100ED0000131013AF4E71AB191F90020981A10BDD6
:100EE0001046FCE703460246D01A12F9011B0029FE
:100EF000FAD1704702440346934202D003F8011B23
:100F0000FAE770472DE9F8431F4D14460746884617
:100F100095F8242052BBDFF870909CB395F82430EC
:100F20002BB92022FF2148462F62FFF7E3FF95F8F7
:100F300024004146C0F1080205EB8000A24228BF10
:100F40002246D6B29200FFF7AFFF95F82430A41BDB
:100F500017441E449044E4B2F6B2082E85F824608B
:100F6000DBD1FFF711FF0028D7D108E02B6A03EB94
:100F700082038342CFD0FFF707FF0028CBD10020A8
:100F8000BDE8F8830120FBE79C230020024B1A7880
:100F9000024B1A70704700BFDC2300201022002093
:100FA000F8B5194C194800F027FF2146174800F002
:100FB0004FFF24684FF47A70154ED4F89020154DE9
:100FC000D2F80438114F43F00203C2F80438FFF797
:100FD0005BFF2046104901F049F8D4F89020042422
:100FE000D2F8043823F00203C2F804384FF4E13396
:100FF000336055F8040BB84202D0314600F05AFE77
:10100000013CF6D1F8BD00BF1C4D0008183400208B
:10101000C423002014220020244D00080C4B70B57E
:101020000C4D04461E780C4B55F826209A420DD0E4
:101030000A4B002118221846FFF75CFF04600146A6
:1010400055F82600BDE8704000F034BE70BD00BF0A
:10105000DC2300201422002018340020C4230020A8
:101060002DE9F04771B6464B01201D68454BB3F89A
:10107000008000231A46194600F08AFA04468020B0
:1010800002F01CF80746002862D0002C60D03E4ECB
:10109000ADB24FF0800A7369284643F0C0637361B4
:1010A000D6F8143143F0C063C6F8143101F08AFE5B
:1010B00005EB080200FB05F34FF4D06C50434FF0F2
:1010C0003D0E984233D93269520144D4D6F81021EA
:1010D000510140D4216803F100628A602268D76020
:1010E0002268C2F804A02268C2F800C0D4F80090B8
:1010F000D9F8002042F00102C9F80020D4F800908D
:10110000D9F8002022F01E02C9F80020D4F800907F
:10111000D9F80020D207FBD494F80C908033616892
:101120000EFA09F20A60CCE7002001F029FF204600
:1011300000F06EFA384601F0F7FF134B5A6942F09F
:10114000C0625A61D3F8142142F0C062C3F814217E
:1011500061B6BDE8F0870D4B9A6A42F400729A625C
:101160009A6A42F400429A6261B60026012001F0B8
:1011700007FFB045D8D9A819013601F03BFEF8E7C2
:1011800098230020DE2300200020005200ED00E024
:1011900030B50A44084D91420DD011F8013B58403A
:1011A000082340F30004013B2C4013F0FF0384EAC2
:1011B0005000F6D1EFE730BD2083B8ED08B5074BFE
:1011C000074A196801F03D01996053680BB19068B6
:1011D0009847BDE8084002F059B800BF000002403F
:1011E000E023002008B5084B1968890901F03D018A
:1011F0008A019A60054AD3680BB110699847BDE827
:10120000084002F043B800BF00000240E023002085
:1012100008B5084B1968090C01F03D010A049A60F1
:10122000054A53690BB190699847BDE8084002F040
:101230002DB800BF00000240E023002008B5084B95
:101240001968890D01F03D018A059A60054AD36944
:101250000BB1106A9847BDE8084002F017B800BF0C
:1012600000000240E023002008B5074B074A5968F8
:1012700001F03D01D960536A0BB1906A9847BDE80F
:10128000084002F003B800BF00000240E023002045
:1012900008B5084B5968890901F03D018A01DA60F7
:1012A000054AD36A0BB1106B9847BDE8084001F0BE
:1012B000EDBF00BF00000240E023002008B5084B4E
:1012C0005968090C01F03D010A04DA60054A536BC4
:1012D0000BB1906B9847BDE8084001F0D7BF00BF45
:1012E00000000240E023002008B5084B5968890D32
:1012F00001F03D018A05DA60054AD36B0BB1106C31
:101300009847BDE8084001F0C1BF00BF000002409F
:10131000E023002008B5074B074A196801F03D019A
:101320009960536C0BB1906C9847BDE8084001F090
:10133000ADBF00BF00040240E023002008B5084B09
:101340001968890901F03D018A019A60054AD36C48
:101350000BB1106D9847BDE8084001F097BF00BF82
:1013600000040240E023002008B5084B1968090C6E
:1013700001F03D010A049A60054A536D0BB1906D6E
:101380009847BDE8084001F081BF00BF000402405B
:10139000E023002008B5084B1968890D01F03D01D4
:1013A0008A059A60054AD36D0BB1106E9847BDE867
:1013B000084001F06BBF00BF00040240E0230020A2
:1013C00008B5074B074A596801F03D01D960536ED3
:1013D0000BB1906E9847BDE8084001F057BF00BFC1
:1013E00000040240E023002008B5084B5968890931
:1013F00001F03D018A01DA60054AD36E0BB1106F2E
:101400009847BDE8084001F041BF00BF000402401A
:10141000E023002008B5084B5968090C01F03D0194
:101420000A04DA60054A536F0BB1906F9847BDE824
:10143000084001F02BBF00BF00040240E023002061
:1014400008B5084B5968890D01F03D018A05DA603D
:10145000054AD36F13B1D2F880009847BDE8084021
:1014600001F014BF00040240E023002000230C49D7
:1014700010B51A460B4C0B6054F82300026001EBC8
:10148000430004334260402BF6D1074A4FF0FF334C
:101490009360D360C2F80834C2F80C3410BD00BFAA
:1014A000E0230020304B0008000002400F28F8B570
:1014B00010D9102810D0112811D0122808D10F24CB
:1014C0000720DFF8C8E00126DEF80050A04208D966
:1014D000002653E00446F4E70F240020F1E7072438
:1014E000FBE706FA00F73D424AD1264C4FEA001CC2
:1014F0003D4304EB00160EEBC000CEF80050C0E9EF
:101500000123FBB273B12048D0F8D83043F0010377
:10151000C0F8D830D0F8003143F00103C0F80031F2
:10152000D0F8003117F47F4F0ED01748D0F8D830DC
:1015300043F00203C0F8D830D0F8003143F0020382
:10154000C0F80031D0F8003154F80C00036823F0E3
:101550001F030360056815F00105FBD104EB0C03C4
:101560003D2493F80CC05F6804FA0CF43C6021241D
:101570000560446112B1987B00F0D0F93046F8BDA7
:101580000130A3E7304B000800440258E02300205C
:1015900010B5302484F31188FFF788FF002383F30C
:1015A000118810BD10B50446807B00F0CDF90123F1
:1015B0001549627B03FA02F20B6823EA0203DAB2EE
:1015C0000B6072B9114AD2F8D81021F00101C2F8AB
:1015D000D810D2F8001121F00101C2F80011D2F8A0
:1015E000002113F47F4F0ED1084BD3F8D82022F0FE
:1015F0000202C3F8D820D3F8002122F00202C3F877
:101600000021D3F8003110BDE0230020004402582F
:1016100008B5302383F31188FFF7C4FF002383F359
:10162000118808BD026843681143016003B118477F
:1016300070470000024A136843F0C003136070470C
:1016400000480040024A136843F0C003136070472B
:1016500000500040024A136843F0C0031360704713
:1016600000780040064BD3F8E8200243C3F8E82096
:10167000D3F810211043C3F81001D3F8103170478C
:101680000044025837B5274C274D204600F006FB92
:1016900004F11400009400234FF40072234900F079
:1016A000C3F94FF40072224904F138000094214B31
:1016B00000F03CFA204BC4E91735204C204600F0DE
:1016C000EDFA04F11400009400234FF400721C4959
:1016D00000F0AAF94FF400721A4904F1380000949E
:1016E000194B00F023FA194BC4E91735184C204662
:1016F00000F0D4FA04F1140000234FF400721549ED
:10170000009400F091F9144B4FF40072134904F166
:101710003800009400F00AFA114BC4E9173503B001
:1017200030BD00BF6424002000E1F505A82500209D
:10173000A82B00203516000800480040D0240020C7
:10174000A8270020A82D00204516000800500040C2
:101750003C250020A829002055160008A82F0020AD
:101760000078004038B5264D0446037C002918BF98
:101770000D46012B06D1234B984230D14FF48020E7
:10178000FFF770FF2A68236EE16D03EB5203A56635
:10179000B3FBF2F36A68100442BF23F0070003F0C2
:1017A000070343EA4003CB60AB6843F040034B6060
:1017B000EB6843F001038B6042F4967343F001033E
:1017C0000B604FF0FF330B62510505D512F010226C
:1017D00011D0B2F1805F10D084F8643038BD0A4B6C
:1017E000984205D0094B9842CCD14FF08040C7E7D2
:1017F0004FF48010C4E77F23EEE73F23ECE700BF00
:10180000304C000864240020D02400203C25002017
:101810002DE9F047C66D05463768F4692107346243
:101820001AD014F0080118BF4FF48071E20748BFC6
:1018300041F02001A3074FF0300348BF41F04001C1
:10184000600748BF41F0800183F31188281DFFF72E
:10185000E9FE002383F31188E2050AD5302383F3E0
:1018600011884FF48061281DFFF7DCFE002383F30D
:1018700011884FF030094FF0000A14F0200838D1D9
:101880003B0616D54FF0300905F1380A200610D571
:1018900089F31188504600F07DF9002836DA0821D6
:1018A000281DFFF7BFFE27F080033360002383F37A
:1018B0001188790614D5620612D5302383F3118876
:1018C000D5E913239A4208D12B6C33B127F0400796
:1018D0001021281DFFF7A6FE3760002383F311882F
:1018E000E30618D5AA6E1369ABB15069BDE8F0479D
:1018F000184789F31188736A284695F864101940CF
:1019000000F0E6F98AF31188F469B6E7B06288F36B
:101910001188F469BAE7BDE8F0870000090100F119
:101920006043012203F56143C9B283F8001300F05C
:101930001F039A4043099B0003F1604303F5614391
:10194000C3F880211A60704700F01F0301229A40FB
:10195000430900F160409B0000F5614003F16043E2
:1019600003F56143C3F88020C3F88021002380F889
:1019700000337047F8B51546826804460B46AA4204
:1019800000D28568A1692669761AB5420BD218463D
:101990002A46FFF789FAA3692B44A3612846A36866
:1019A0005B1BA360F8BD0CD9AF1B18463246FFF78E
:1019B0007BFA3A46E1683044FFF776FAE3683B4445
:1019C000EBE718462A46FFF76FFAE368E5E7000001
:1019D00083689342F7B50446154600D28568D4E97A
:1019E0000460361AB5420BD22A46FFF75DFA6369E6
:1019F0002B4463612846A3685B1BA36003B0F0BD62
:101A00000DD93246AF1B0191FFF74EFA01993A46C4
:101A1000E0683144FFF748FAE3683B44E9E72A46C7
:101A2000FFF742FAE368E4E710B50A440024C36113
:101A3000029B8460C16002610362C0E90000C0E9EA
:101A4000051110BD08B5D0E90532934201D1826875
:101A500082B98268013282605A1C42611970002189
:101A6000D0E904329A4224BFC368436100F0B0FE5B
:101A7000002008BD4FF0FF30FBE7000070B53023B9
:101A800004460E4683F31188A568A5B1A368A26930
:101A9000013BA360531CA36115782269934224BFC4
:101AA000E368A361E3690BB120469847002383F301
:101AB0001188284607E03146204600F079FE0028CC
:101AC000E2DA85F3118870BD2DE9F74F04460E4622
:101AD00017469846D0F81C904FF0300A8AF31188C8
:101AE0004FF0000B154665B12A4631462046FFF7F8
:101AF00041FF034660B94146204600F059FE0028E8
:101B0000F1D0002383F31188781B03B0BDE8F08F78
:101B1000B9F1000F03D001902046C847019B8BF319
:101B20001188ED1A1E448AF31188DCE7C160C36195
:101B3000009B82600362C0E905111144C0E9000006
:101B400001617047F8B504460D461646302383F30D
:101B50001188A768A7B1A368013BA36063695A1CF9
:101B600062611D70D4E904329A4224BFE368636164
:101B7000E3690BB120469847002080F3118807E005
:101B80003146204600F014FE0028E2DA87F311887F
:101B9000F8BD0000D0E9052310B59A4201D1826852
:101BA0007AB982680021013282605A1C82611C78F5
:101BB00003699A4224BFC368836100F009FE20468E
:101BC00010BD4FF0FF30FBE72DE9F74F04460E46FE
:101BD00017469846D0F81C904FF0300A8AF31188C7
:101BE0004FF0000B154665B12A4631462046FFF7F7
:101BF000EFFE034660B94146204600F0D9FD0028BB
:101C0000F1D0002383F31188781B03B0BDE8F08F77
:101C1000B9F1000F03D001902046C847019B8BF318
:101C20001188ED1A1E448AF31188DCE702684368C4
:101C30001143016003B11847704700001430FFF7EB
:101C400043BF00004FF0FF331430FFF73DBF0000EB
:101C50003830FFF7B9BF00004FF0FF333830FFF7DF
:101C6000B3BF00001430FFF709BF00004FF0FF3191
:101C70001430FFF703BF00003830FFF763BF0000E8
:101C80004FF0FF323830FFF75DBF0000012914BF6D
:101C90006FF0130000207047FFF7F4BC044B0360A3
:101CA00000234360C0E9023301230374704700BF7F
:101CB000484C000810B53023044683F31188FFF721
:101CC00051FD02230020237480F3118810BD000011
:101CD00038B5C36904460D461BB904210844FFF713
:101CE000A5FF294604F11400FFF7ACFE002806DA30
:101CF000201D4FF40061BDE83840FFF797BF38BDA5
:101D0000026843681143016003B11847704700003F
:101D100013B5406B00F58054D4F8A4381A681178D4
:101D2000042914D1017C022911D1197901231289C6
:101D30008B4013420BD101A94C3002F097F9D4F833
:101D4000A4480246019B2179206800F0DFF902B027
:101D500010BD0000143002F019B900004FF0FF333D
:101D6000143002F013B900004C3002F0EBB900005F
:101D70004FF0FF334C3002F0E5B90000143002F0B0
:101D8000E7B800004FF0FF31143002F0E1B8000076
:101D90004C3002F0B7B900004FF0FF324C3002F087
:101DA000B1B900000020704710B500F58054D4F898
:101DB000A4381A681178042917D1017C022914D19A
:101DC0005979012352898B4013420ED1143002F00D
:101DD00079F8024648B1D4F8A4484FF440736179C9
:101DE0002068BDE8104000F07FB910BD406BFFF7E0
:101DF000DBBF0000704700007FB5124B01250426B1
:101E0000044603600023057400F184024360294600
:101E1000C0E902330C4B0290143001934FF440732D
:101E2000009602F02BF8094B04F69442294604F17F
:101E30004C000294CDE900634FF4407302F0F2F8D5
:101E400004B070BD704C0008ED1D0008111D0008A5
:101E50000A68302383F311880B790B3342F823008F
:101E60004B79133342F823008B7913B10B3342F8CB
:101E7000230000F58053C3F8A41802230374002044
:101E800080F311887047000038B5037F044613B112
:101E900090F85430ABB90125201D0221FFF730FF27
:101EA00004F114006FF00101257700F09DFC04F1AE
:101EB0004C0084F854506FF00101BDE8384000F048
:101EC00093BC38BD10B5012104460430FFF718FF5C
:101ED0000023237784F8543010BD000038B5044641
:101EE0000025143001F0E2FF04F14C00257702F0E8
:101EF000B1F8201D84F854500121FFF701FF20465E
:101F0000BDE83840FFF750BF90F8803003F0600321
:101F1000202B06D190F881200023212A03D81F2AE4
:101F200006D800207047222AFBD1C0E91D3303E008
:101F3000034A426707228267C3670120704700BFD8
:101F40003C22002037B500F58055D5F8A4381A6832
:101F5000117804291AD1017C022917D1197901239A
:101F600012898B40134211D100F14C04204602F03B
:101F700031F958B101A9204602F078F8D5F8A44803
:101F80000246019B2179206800F0C0F803B030BD03
:101F900001F10B03F0B550F8236085B004460D46FF
:101FA000FEB1302383F3118804EB8507301D08212F
:101FB000FFF7A6FEFB6806F14C005B691B681BB1CE
:101FC000019002F061F8019803A902F04FF802466F
:101FD00048B1039B2946204600F098F8002383F37C
:101FE000118805B0F0BDFB685A691268002AF5D067
:101FF0001B8A013B1340F1D104F18002EAE70000A3
:10200000133138B550F82140ECB1302383F31188F7
:1020100004F58053D3F8A4281368527903EB8203A4
:10202000DB689B695D6845B104216018FFF768FEB5
:10203000294604F1140001F04FFF2046FFF7B4FEDB
:10204000002383F3118838BD7047000001F01CBAEB
:1020500001234022002110B5044600F8303BFEF772
:1020600049FF0023C4E9013310BD000010B530233F
:10207000044683F311882422416000210C30FEF7CE
:1020800039FF204601F022FA02230020237080F35A
:10209000118810BD70B500EB8103054650690E46EE
:1020A0001446DA6018B110220021FEF723FFA06960
:1020B00018B110220021FEF71DFF31462846BDE869
:1020C000704001F009BB000083682022002103F06A
:1020D000011310B5044683601030FEF70BFF204655
:1020E000BDE8104001F084BBF0B4012500EB810491
:1020F00047898D40E4683D43A469458123600023FE
:10210000A2606360F0BC01F0A1BB0000F0B4012547
:1021100000EB810407898D40E4683D4364690581D3
:1021200023600023A2606360F0BC01F017BC0000D4
:1021300070B5022300250446242203702946C0F806
:1021400088500C3040F8045CFEF7D4FE204684F83A
:10215000705001F055FA63681B6823B12946204688
:10216000BDE87040184770BD0378052B10B50446D4
:102170000AD080F88C300523037043681B680BB1CC
:10218000042198470023A36010BD000001780529B1
:1021900006D190F88C20436802701B6803B1184781
:1021A0007047000070B590F87030044613B10023FA
:1021B00080F8703004F18002204601F03DFB636836
:1021C0009B68B3B994F8803013F0600535D00021D6
:1021D000204601F02FFE0021204601F01FFE63681B
:1021E0001B6813B1062120469847062384F87030F7
:1021F00070BD204698470028E4D0B4F88630A26F1E
:102200009A4288BFA36794F98030A56F002B4FF0E6
:10221000300380F20381002D00F0F280092284F85F
:10222000702083F3118800212046D4E91D23FFF795
:102230006DFF002383F31188DAE794F8812003F01F
:102240007F0343EA022340F20232934200F0C5804A
:1022500021D8B3F5807F48D00DD8012B3FD0022B79
:1022600000F09380002BB2D104F188026267022251
:10227000A267E367C1E7B3F5817F00F09B80B3F508
:10228000407FA4D194F88230012BA0D1B4F88830DB
:1022900043F0020332E0B3F5006F4DD017D8B3F529
:1022A000A06F31D0A3F5C063012B90D8636820469E
:1022B00094F882205E6894F88310B4F88430B047B4
:1022C000002884D0436863670368A3671AE0B3F506
:1022D000106F36D040F6024293427FF478AF5C4BE9
:1022E00063670223A3670023C3E794F88230012BBE
:1022F0007FF46DAFB4F8883023F00203A4F888307F
:10230000C4E91D55E56778E7B4F88030B3F5A06FF0
:102310000ED194F88230204684F88A3001F0CEF94C
:1023200063681B6813B1012120469847032323707B
:102330000023C4E91D339CE704F18B036367012389
:10234000C3E72378042B10D1302383F31188204670
:10235000FFF7BAFE85F311880321636884F88B5078
:1023600021701B680BB12046984794F88230002BEF
:10237000DED084F88B300423237063681B68002B45
:10238000D6D0022120469847D2E794F884302046E0
:102390001D0603F00F010AD501F040FA012804D010
:1023A00002287FF414AF2B4B9AE72B4B98E701F0F0
:1023B00027FAF3E794F88230002B7FF408AF94F803
:1023C000843013F00F01B3D01A06204602D501F075
:1023D00049FDADE701F03AFDAAE794F88230002B01
:1023E0007FF4F5AE94F8843013F00F01A0D01B06F3
:1023F000204602D501F01EFD9AE701F00FFD97E798
:10240000142284F8702083F311882B462A4629462B
:102410002046FFF769FE85F31188E9E65DB11522D4
:1024200084F8702083F3118800212046D4E91D230D
:10243000FFF75AFEFDE60B2284F8702083F3118823
:102440002B462A4629462046FFF760FEE3E700BFF9
:10245000A04C0008984C00089C4C000838B590F837
:1024600070300446002B3ED0063BDAB20F2A34D837
:102470000F2B32D8DFE803F0373131082232313107
:102480003131313131313737856FB0F886309D4287
:1024900014D2C3681B8AB5FBF3F203FB12556DB966
:1024A000302383F311882B462A462946FFF72EFE58
:1024B00085F311880A2384F870300EE0142384F821
:1024C0007030302383F31188002320461A461946C2
:1024D000FFF70AFE002383F3118838BDC36F03B1F1
:1024E00098470023E7E70021204601F0A3FC0021E4
:1024F000204601F093FC63681B6813B10621204657
:1025000098470623D7E7000010B590F870300446CE
:10251000142B29D017D8062B05D001D81BB110BD1C
:10252000093B022BFBD80021204601F083FC00214F
:10253000204601F073FC63681B6813B10621204636
:102540009847062319E0152BE9D10B2380F870304A
:10255000302383F3118800231A461946FFF7D6FD6E
:10256000002383F31188DAE7C3689B695B68002B5B
:10257000D5D1C36F03B19847002384F87030CEE7FC
:1025800000238268037503691B6899689142FBD236
:102590005A68036042601060586070470023826888
:1025A000037503691B6899689142FBD85A680360F8
:1025B000426010605860704708B50846302383F3C6
:1025C00011880A7D0023052A06D8DFE802F00B05F2
:1025D0000503120E826913604FF0FF338361FFF72A
:1025E000CFFF002383F3118808BD8269936801330C
:1025F0009360D0E9003213605A60EDE7FFF7C0BF87
:10260000054BD96808751868026853601A60012282
:10261000D8600275FDF7F6BEA83100200C4B30B52E
:10262000DD684B1C87B004460FD02B46094A68462C
:1026300000F06EF92046FFF7E3FF009B13B16846F8
:1026400000F070F9A86907B030BDFFF7D9FFF9E7CE
:10265000A8310020B925000838B50C4D0446816129
:10266000EB6881689A68914203D8BDE83840FFF76B
:1026700087BF1846FFF792FF01230146EC60204612
:102680002375BDE83840FDF7BDBE00BFA83100206E
:10269000044B1A68DB6890689B68984294BF0020DE
:1026A00001207047A8310020084B10B51C68D8687D
:1026B000226853601A600122DC602275FFF76EFF0A
:1026C00001462046BDE81040FDF79CBEA831002021
:1026D00038B50123084C00252370656001F0B6FD74
:1026E00001F0DCFD0549064801F0B0FE022323702D
:1026F00085F3118838BD00BF10340020A84C0008B5
:10270000A831002000F044B9034A516853685B1AAD
:102710009842FBD8704700BF001000E08B60022396
:10272000086108468B8270478368A3F1840243F8EE
:10273000142C026943F8442C426943F8402C094A9E
:1027400043F8242CC268A3F1200043F8182C02227D
:1027500003F80C2C002203F80B2C034A43F8102C2E
:10276000704700BF1D040008A831002008B5FFF71E
:10277000DBFFBDE80840FFF741BF0000024BDB680C
:1027800098610F20FFF73CBFA8310020302383F36E
:102790001188FFF7F3BF000008B50146302383F32B
:1027A00011880820FFF73AFF002383F3118808BD42
:1027B000064BDB6839B1426818605A6013604360A9
:1027C0000420FFF72BBF4FF0FF307047A8310020E7
:1027D0000368984206D01A680260506018469961F2
:1027E000FFF70CBF7047000038B504460D4620685F
:1027F000844200D138BD036823605C608561FFF7C7
:10280000FDFEF4E7036810B59C68A2420CD85C6832
:102810008A600B604C602160596099688A1A9A60DE
:102820004FF0FF33836010BD121B1B68ECE7000004
:102830000A2938BF0A2170B504460D460A266019D8
:1028400001F0FEFC01F0E6FC041BA54203D8751C58
:1028500004462E46F3E70A2E04D90120BDE8704055
:1028600001F034BE70BD0000F8B5144B0D460A2AC5
:102870004FF00A07D96103F11001826038BF0A22C4
:10288000416019691446016048601861A81801F098
:10289000C7FC01F0BFFC431B0646A34206D37C1CC9
:1028A00028192746354601F0CBFCF2E70A2F04D958
:1028B0000120BDE8F84001F009BEF8BDA8310020B4
:1028C000F8B506460D4601F0A5FC0F4A134653F82D
:1028D000107F9F4206D12A4601463046BDE8F840A7
:1028E000FFF7C2BFD169BB68441A2C1928BF2C4618
:1028F000A34202D92946FFF79BFF224631460348EF
:10290000BDE8F840FFF77EBFA8310020B8310020B5
:10291000C0E90323002310B45DF8044B4361FFF7C3
:10292000CFBF000010B5194C236998420DD08168C3
:10293000D0E9003213605A609A680A449A60002312
:1029400003604FF0FF33A36110BD0268234643F8D4
:10295000102F53600022026022699A4203D1BDE821
:10296000104001F067BC936881680B44936001F0EC
:1029700051FC2269E1699268441AA242E4D91144E7
:10298000BDE81040091AFFF753BF00BFA83100206F
:102990002DE9F047DFF8BC8008F110072C4ED8F87D
:1029A000105001F037FCD8F81C40AA68031B9A426B
:1029B0003ED814444FF00009D5E90032C8F81C4055
:1029C00013605A60C5F80090D8F81030B34201D1B6
:1029D00001F030FC89F31188D5E903312846984786
:1029E000302383F311886B69002BD8D001F012FCDF
:1029F0006A69A0EB040982464A450DD2022001F023
:102A000065FD0022D8F81030B34208D1514628465F
:102A1000BDE8F047FFF728BF121A2244F2E712EB95
:102A200009092946384638BF4A46FFF7EBFEB5E7A5
:102A3000D8F81030B34208D01444C8F81C00211A4A
:102A4000A960BDE8F047FFF7F3BEBDE8F08700BF1F
:102A5000B8310020A831002000207047FEE70000B8
:102A6000704700004FF0FF307047000002290CD083
:102A7000032904D00129074818BF00207047032A02
:102A800005D8054800EBC200704704487047002095
:102A9000704700BF804D00084C220020344D0008D4
:102AA00070B59AB005460846144601A900F0C2F870
:102AB00001A8FEF717FA431C0022C6B25B001046BD
:102AC000C5E9003423700323023404F8013C01AB50
:102AD000D1B202348E4201D81AB070BD13F8011B76
:102AE000013204F8010C04F8021CF1E708B53023A8
:102AF00083F311880348FFF725FA002383F3118835
:102B000008BD00BF1834002090F8803003F01F0289
:102B1000012A07D190F881200B2A03D10023C0E9B4
:102B20001D3315E003F06003202B08D1B0F884308A
:102B30002BB990F88120212A03D81F2A04D8FFF747
:102B4000E3B9222AEBD0FAE7034A426707228267F9
:102B5000C3670120704700BF4322002007B5052945
:102B600017D8DFE801F0191603191920302383F371
:102B70001188104A01210190FFF78CFA0198022177
:102B80000D4AFFF787FA0D48FFF7A8F9002383F3F2
:102B9000118803B05DF804FB302383F311880748E4
:102BA000FFF772F9F2E7302383F311880348FFF748
:102BB00089F9EBE7D44C0008F84C000818340020E1
:102BC00038B50C4D0C4C2A460C4904F10800FFF7AF
:102BD00067FF05F1CA0204F110000949FFF760FF21
:102BE00005F5CA7204F118000649BDE83840FFF740
:102BF00057BF00BFF04C00204C220020B44C00080E
:102C0000BE4C0008C94C000870B5044608460D4685
:102C1000FEF768F9C6B22046013403780BB91846AE
:102C200070BD32462946FEF749F90028F3D101204C
:102C3000F6E700002DE9F84F05460C46FEF752F97D
:102C40002A49C6B22846FFF7DFFF08B1013EF6B2B7
:102C500027492846FFF7D8FF08B11036F6B2632E91
:102C60000DD8DFF88890DFF888A0224FDFF88CB00D
:102C7000DFF88C802E7846B92670BDE8F88F29469B
:102C80002046BDE8F84F01F01DBF252E2AD10722AE
:102C900049462846FEF712F950B9D8F800300735F2
:102CA000063444F8063CB8F8043024F8023CE1E766
:102CB000082251462846FEF701F998B9A21C0E4B8E
:102CC000197802320909C95D02F8041C13F8011BC6
:102CD00001F00F015B45C95D02F8031CF0D1183407
:102CE0000835C7E7013504F8016BC3E7A04D0008BC
:102CF000C94C0008AF4D000800E8F11F0CE8F11FB7
:102D0000A84D0008BFF34F8F044B1A695107FCD13F
:102D1000D3F810215207F8D1704700BF00200052AD
:102D200008B50D4B1B78ABB9FFF7ECFF0B4BDA681E
:102D3000D10704D50A4A5A6002F188325A60D3F8A2
:102D40000C21D20706D5064AC3F8042102F18832C5
:102D5000C3F8042108BD00BF4E4F002000200052E0
:102D60002301674508B5114B1B78F3B9104B1A695D
:102D7000510703D5DA6842F04002DA60D3F8102137
:102D8000520705D5D3F80C2142F04002C3F80C21BC
:102D9000FFF7B8FF064BDA6842F00102DA60D3F8B9
:102DA0000C2142F00102C3F80C2108BD4E4F002057
:102DB000002000520F289ABF00F5806040040020D8
:102DC000704700004FF4003070470000102070473B
:102DD0000F2808B50BD8FFF7EDFF00F500330268A8
:102DE000013204D104308342F9D1012008BD002012
:102DF000FCE700000F2838B505463FD8FFF782FFF3
:102E00001F4CFFF78DFF4FF0FF3307286361C4F8B5
:102E100014311DD82361FFF775FF030243F024032B
:102E2000E360E36843F08003E36023695A07FCD45E
:102E30002846FFF767FFFFF7BDFF4FF4003100F0B2
:102E4000C5F92846FFF78EFFBDE83840FFF7C0BF41
:102E5000C4F81031FFF756FFA0F108031B0243F03E
:102E60002403C4F80C31D4F80C3143F08003C4F8C7
:102E70000C31D4F810315B07FBD4D9E7002038BD02
:102E8000002000522DE9F84F04460D46104644EA52
:102E90000203DE0602D00020BDE8F88F20F01F00FC
:102EA000DFF8D4B0DFF8D4A0FFF73AFF05EB000855
:102EB000454503D10120FFF755FFEDE720222946C4
:102EC000204601F0EFFD10B920342035F0E723460D
:102ED00004F120021F68791CDDD104339342F9D13B
:102EE00004F178432048214EB3F5801F204B38BFB2
:102EF000184603F1F80332BFD946D1461E46FFF704
:102F000001FF0760A4EB050C336805F11C0143F0D9
:102F1000020333602B1FD9F8007017F00507FAD1B0
:102F200053F8042F8B424CF80320F4D1BFF34F8F9A
:102F3000FFF7E8FE4FF0FF330360336823F002032E
:102F40003360BFF34F8F0B4BC3F85C42BFF34F8F1F
:102F5000BFF36F8F20222946204601F0A3FD0028F1
:102F6000B2D03846A7E700BF142100520C2000520F
:102F70001420005200ED00E01020005210210052F9
:102F800010B5084C237828B11BB9FFF7C9FE0123FF
:102F9000237010BD002BFCD02070BDE81040FFF75F
:102FA000E1BE00BF4E4F00202DE9F04F0D4685B029
:102FB000814658B111F00D0614BF2022082211F0ED
:102FC0000803019304D0431E03426AD0002435E075
:102FD000002E37D009F11F0121F01F094FF0010821
:102FE000324F05F00403DFF8D0A005EA080BBBF16F
:102FF000000F32D07869C0072FD408F101080C37D0
:10300000B8F1060FF3D19EB9294D4946A81901928E
:1030100001F066F9044600283AD11836019A782E54
:10302000F3D1494601F05CF90446002830D1019AF9
:103030004946204801F054F9044668BB204605B0D3
:10304000BDE8F08F0029C9D101462846029201F05F
:1030500047F90446E0B9029AC0E713B1786941071D
:10306000CBD5AC0702D578698007C6D5019911B1D7
:1030700078690107C1D51820494600FB08A0CDE9B1
:10308000022301F02DF90446DDE902230028B4D023
:103090004A460021204601E04A460021FDF72AFF6A
:1030A000CCE70246002E95D198E700BFC04D00083E
:1030B000804F0020504F0020684F00200121FFF773
:1030C00073BF0000F8B500231A461A600433B3F545
:1030D000806FFAD1114D01241827114E07FB0460AF
:1030E00001342A6955F80C1F01F0E6F8062CF5D1D9
:1030F00037254FF4C0542046FFF7E0FF014628B1C2
:1031000022460848BDE8F84001F0D6B8C4EBC40434
:10311000013D4FEAD404EED1F8BD00BFC04D000818
:10312000684F0020504F002008B101F04BB97047A4
:103130000244074BD2B210B5904200D110BD441CDE
:1031400000B253F8200041F8040BE0B2F4E700BFEE
:10315000504000580E4B30B51C6F240405D41C6F32
:103160001C671C6F44F400441C670A4C024423682B
:10317000D2B243F480732360074B904200D130BD3C
:10318000441C51F8045B00B243F82050E0B2F4E76D
:1031900000440258004802585040005807B5012228
:1031A00001A90020FFF7C4FF019803B05DF804FBFC
:1031B00013B50446FFF7F2FFA04205D0012201A992
:1031C00000200194FFF7C6FF02B010BD0144BFF319
:1031D0004F8F064B884204D3BFF34F8FBFF36F8FDF
:1031E0007047C3F85C022030F4E700BF00ED00E058
:1031F000034B1A681AB9034AD2F8D0241A607047F0
:10320000F84F00200040025808B5FFF7F1FF024BCD
:103210001868C0F3806008BDF84F0020EFF3098301
:10322000054968334A6B22F001024A6383F3098837
:10323000002383F31188704700EF00E0302080F313
:10324000118862B60D4B0E4AD96821F4E061090479
:10325000090C0A430B49DA60D3F8FC2042F0807273
:10326000C3F8FC20084AC2F8B01F116841F0010100
:1032700011602022DA7783F82200704700ED00E029
:103280000003FA0555CEACC5001000E0302310B5A0
:1032900083F311880E4B5B6813F4006314D0F1EED6
:1032A000103AEFF309844FF08073683CE361094BF7
:1032B000DB6B236684F30988FFF7EAF910B1064B4C
:1032C000A36110BD054BFBE783F31188F9E700BF4D
:1032D00000ED00E000EF00E02F04000832040008D9
:1032E00070B5BFF34F8FBFF36F8F1A4A0021C2F83A
:1032F0005012BFF34F8FBFF36F8F536943F4003306
:103300005361BFF34F8FBFF36F8FC2F88410BFF3C9
:103310004F8FD2F8803043F6E074C3F3C900C3F393
:103320004E335B0103EA0406014646EA8175013922
:10333000C2F86052F9D2203B13F1200FF2D1BFF353
:103340004F8F536943F480335361BFF34F8FBFF303
:103350006F8F70BD00ED00E0FEE70000214B2248BA
:10336000224A70B5904237D3214BC11EDA1C121A83
:1033700022F003028B4238BF00220021FDF7BAFD84
:103380001C4A0023C2F88430BFF34F8FD2F880303C
:1033900043F6E074C3F3C900C3F34E335B0103EAA1
:1033A0000406014646EA81750139C2F86C52F9D229
:1033B000203B13F1200FF2D1BFF34F8FBFF36F8F7C
:1033C000BFF34F8FBFF36F8F0023C2F85032BFF3AC
:1033D0004F8FBFF36F8F70BD53F8041B40F8041B71
:1033E000C0E700BFF44F00086C5100206C51002072
:1033F0006C51002000ED00E0074BD3F8D81021EA13
:103400000001C3F8D810D3F8002122EA0002C3F863
:103410000021D3F8003170470044025870B5D0E95C
:10342000244300224FF0FF359E6804EB4213510104
:10343000D3F80009002805DAD3F8000940F08040ED
:10344000C3F80009D3F8000B002805DAD3F8000B05
:1034500040F08040C3F8000B013263189642C3F875
:103460000859C3F8085BE0D24FF00113C4F81C38C8
:1034700070BD0000890141F02001016103699B06D4
:10348000FCD41220FFF740B910B50A4C2046FEF7D5
:10349000DFFD094BC4F89030084BC4F89430084C59
:1034A0002046FEF7D5FD074BC4F89030064BC4F814
:1034B000943010BDFC4F0020000008402C4E000846
:1034C0009850002000000440384E000870B5037882
:1034D0000546012B5CD1434BD0F89040984258D11F
:1034E000414B0E216520D3F8D82042F00062C3F88A
:1034F000D820D3F8002142F00062C3F80021D3F8AD
:103500000021D3F8802042F00062C3F88020D3F875
:10351000802022F00062C3F88020D3F88030FEF7CC
:10352000FDF9324BE360324BC4F800380023D5F884
:103530009060C4F8003EC02323604FF40413A363DB
:103540003369002BFCDA01230C203361FFF7DCF830
:103550003369DB07FCD41220FFF7D6F83369002B60
:10356000FCDA00262846A660FFF758FF6B68C4F80F
:103570001068DB68C4F81468C4F81C6883BB1D4B72
:10358000A3614FF0FF336361A36843F00103A360BD
:1035900070BD194B9842C9D1134B4FF08060D3F8DE
:1035A000D82042F00072C3F8D820D3F8002142F0AE
:1035B0000072C3F80021D3F80021D3F8802042F034
:1035C0000072C3F88020D3F8802022F00072C3F884
:1035D0008020D3F88030FFF70FFF0E214D209EE7AB
:1035E000064BCDE7FC4F0020004402584014004039
:1035F00003002002003C30C098500020083C30C03E
:10360000F8B5D0F89040054600214FF000662046FE
:10361000FFF730FFD5F8941000234FF001128F68A8
:103620004FF0FF30C4F83438C4F81C2804EB4312C0
:1036300001339F42C2F80069C2F8006BC2F8080962
:10364000C2F8080BF2D20B68D5F89020C5F8983074
:10365000636210231361166916F01006FBD1122065
:10366000FFF752F8D4F8003823F4FE63C4F80038AA
:10367000A36943F4402343F01003A3610923C4F872
:103680001038C4F814380B4BEB604FF0C043C4F84B
:10369000103B094BC4F8003BC4F81069C4F800396A
:1036A000D5F8983003F1100243F48013C5F8982040
:1036B000A362F8BD084E000840800010D0F89020AA
:1036C00090F88A10D2F8003823F4FE6343EA01131D
:1036D000C2F80038704700002DE9F84300EB810381
:1036E000D0F890500C468046DA680FFA81F948010C
:1036F000166806F00306731E022B05EB41134FF00C
:10370000000194BFB604384EC3F8101B4FF00101FE
:1037100004F1100398BF06F1805601FA03F3916992
:1037200098BF06F5004600293AD0578A04F158019F
:10373000374349016F50D5F81C180B430021C5F8D9
:103740001C382B180127C3F81019A7405369611EB4
:103750009BB3138A928B9B08012A88BF5343D8F8E6
:103760009820981842EA034301F140022146C8F824
:103770009800284605EB82025360FFF77BFE08EBBA
:103780008900C3681B8A43EA845348341E4364019A
:103790002E51D5F81C381F43C5F81C78BDE8F883B6
:1037A00005EB4917D7F8001B21F40041C7F8001BAF
:1037B000D5F81C1821EA0303C0E704F13F030B4AC4
:1037C0002846214605EB83035A60FFF753FE05EBBD
:1037D0004910D0F8003923F40043C0F80039D5F877
:1037E0001C3823EA0707D7E7008000100004000216
:1037F000D0F894201268C0F89820FFF70FBE0000A0
:103800005831D0F8903049015B5813F4004004D08F
:1038100013F4001F0CBF0220012070474831D0F87C
:10382000903049015B5813F4004004D013F4001F9A
:103830000CBF02200120704700EB8101CB68196AA0
:103840000B6813604B6853607047000000EB810306
:1038500030B5DD68AA691368D36019B9402B84BFFD
:10386000402313606B8A1468D0F890201C4402EB4C
:103870004110013C09B2B4FBF3F46343033323F07A
:10388000030343EAC44343F0C043C0F8103B2B6832
:1038900003F00303012B0ED1D2F8083802EB4110DC
:1038A00013F4807FD0F8003B14BF43F0805343F003
:1038B0000053C0F8003B02EB4112D2F8003B43F04A
:1038C0000443C2F8003B30BD2DE9F041D0F89060D0
:1038D00005460C4606EB4113D3F8087B3A07C3F8BC
:1038E000087B08D5D6F814381B0704D500EB8103F4
:1038F000DB685B689847FA071FD5D6F81438DB07F2
:103900001BD505EB8403D968CCB98B69488A5A6802
:10391000B2FBF0F600FB16228AB91868DA6890420A
:103920000DD2121AC3E90024302383F311882146F3
:103930002846FFF78BFF84F31188BDE8F08101234F
:1039400003FA04F26B8923EA02036B81CB68002B34
:10395000F3D021462846BDE8F041184700EB81032B
:103960004A0170B5DD68D0F890306C692668E66071
:1039700056BB1A444FF40020C2F810092A6802F01E
:103980000302012A0AB20ED1D3F8080803EB42144D
:1039900010F4807FD4F8000914BF40F0805040F04C
:1039A0000050C4F8000903EB4212D2F8000940F0BD
:1039B0000440C2F800090122D3F8340802FA01F1E8
:1039C0000143C3F8341870BD19B9402E84BF40209C
:1039D000206020681A442E8A8419013CB4FBF6F456
:1039E00040EAC44040F00050C6E700002DE9F8432B
:1039F000D0F8906005460C464F0106EB4113D3F812
:103A0000088918F0010FC3F808891CD0D6F81038BF
:103A1000DB0718D500EB8103D3F80CC0DCF81430B9
:103A2000D3F800E0DA68964530D2A2EB0E024FF0F0
:103A300000091A60C3F80490302383F31188FFF75C
:103A40008DFF89F3118818F0800F1DD0D6F8343817
:103A50000126A640334217D005EB84030134D5F884
:103A60009050D3F80CC0E4B22F44DCF8142005EBDE
:103A70000434D2F800E05168714514D3D5F83438D5
:103A800023EA0606C5F83468BDE8F883012303FA83
:103A900001F2038923EA02030381DCF80830002BDA
:103AA000D1D09847CFE7AEEB0103BCF810008342BA
:103AB00028BF0346D7F8180980B2B3EB800FE3D8CC
:103AC0009068A0F1040959F8048FC4F80080A0EBB5
:103AD00009089844B8F1040FF5D818440B449060D5
:103AE0005360C8E72DE9F84FD0F8905004466E694E
:103AF000AB691E4016F480586E6103D0BDE8F84FE4
:103B0000FEF716BB002E12DAD5F8003E9B0705D053
:103B1000D5F8003E23F00303C5F8003ED5F804387D
:103B2000204623F00103C5F80438FEF72FFB3705C4
:103B300005D52046FFF772FC2046FEF715FBB004C2
:103B40000CD5D5F8083813F0060FEB6823F4705342
:103B50000CBF43F4105343F4A053EB6031071BD563
:103B60006368DB681BB9AB6923F00803AB6123789A
:103B7000052B0CD1D5F8003E9A0705D0D5F8003EAC
:103B800023F00303C5F8003E2046FEF7FFFA636802
:103B9000DB680BB120469847F30200F1BA80B70208
:103BA00026D5D4F8909000274FF0010A09EB471270
:103BB000D2F8003B03F44023B3F5802F11D1D2F8A3
:103BC000003B002B0DDA62890AFA07F322EA0303AD
:103BD000638104EB8703DB68DB6813B13946204659
:103BE00098470137D4F89430FFB29B689F42DDD9E3
:103BF000F00619D5D4F89000026AC2F30A1702F051
:103C00000F0302F4F012B2F5802F00F0CA80B2F573
:103C1000402F09D104EB8303002200F58050DB68BC
:103C20001B6A974240F0B0803003D5F8185835D55C
:103C3000E90303D500212046FFF746FEAA0303D57A
:103C400001212046FFF740FE6B0303D502212046E9
:103C5000FFF73AFE2F0303D503212046FFF734FE7A
:103C6000E80203D504212046FFF72EFEA90203D562
:103C700005212046FFF728FE6A0203D506212046CB
:103C8000FFF722FE2B0203D507212046FFF71CFE7B
:103C9000EF0103D508212046FFF716FE700340F11F
:103CA000A780E90703D500212046FFF79FFEAA075A
:103CB00003D501212046FFF799FE6B0703D50221AA
:103CC0002046FFF793FE2F0703D503212046FFF779
:103CD0008DFEEE0603D504212046FFF787FEA806D9
:103CE00003D505212046FFF781FE690603D506218D
:103CF0002046FFF77BFE2A0603D507212046FFF763
:103D000075FEEB0574D520460821BDE8F84FFFF796
:103D10006DBED4F890904FF0000B4FF0010AD4F82C
:103D200094305FFA8BF79B689F423FF638AF09EB00
:103D30004713D3F8002902F44022B2F5802F20D196
:103D4000D3F80029002A1CDAD3F8002942F0904267
:103D5000C3F80029D3F80029002AFBDB3946D4F840
:103D60009000FFF787FB22890AFA07F322EA030390
:103D7000238104EB8703DB689B6813B13946204637
:103D800098470BF1010BCAE7910701D1D0F80080E9
:103D9000072A02F101029CBF03F8018B4FEA1828A1
:103DA0003FE704EB830300F58050DA68D2F818C0CF
:103DB000DCF80820DCE9001CA1EB0C0C00218F4290
:103DC00008D1DB689B699A683A449A605A683A4419
:103DD0005A6029E711F0030F01D1D0F800808C451B
:103DE00001F1010184BF02F8018B4FEA1828E6E7D0
:103DF000BDE8F88F08B50348FFF774FEBDE808403A
:103E0000FFF744BAFC4F002008B50348FFF76AFEED
:103E1000BDE80840FFF73ABA98500020D0F890303B
:103E200003EB4111D1F8003B43F40013C1F8003B10
:103E300070470000D0F8903003EB4111D1F8003901
:103E400043F40013C1F8003970470000D0F89030F7
:103E500003EB4111D1F8003B23F40013C1F8003B00
:103E600070470000D0F8903003EB4111D1F80039D1
:103E700023F40013C1F800397047000030B5043353
:103E8000039C0172002104FB0325C160C0E90653B5
:103E9000049B0363059BC0E90000C0E90422C0E95C
:103EA0000842C0E90A11436330BD00000022416AA4
:103EB000C260C0E90411C0E90A226FF00101FEF7F7
:103EC00093BC0000D0E90432934201D1C2680AB920
:103ED000181D704700207047036919600021C268EF
:103EE0000132C260C269134482699342036124BFF4
:103EF000436A0361FEF76CBC38B504460D46E368BF
:103F00003BB162690020131D1268A3621344E3628F
:103F100007E0237A33B929462046FEF749FC0028FA
:103F2000EDDA38BD6FF00100FBE70000C368C2693D
:103F3000013BC3604369134482699342436124BFD8
:103F4000436A436100238362036B03B118477047E0
:103F500070B53023044683F31188866A3EB9FFF7B3
:103F6000CBFF054618B186F31188284670BDA36AB9
:103F7000E26A13F8015B9342A36202D32046FFF783
:103F8000D5FF002383F31188EFE700002DE9F84FF8
:103F900004460E46174698464FF0300989F31188BB
:103FA0000025AA46D4F828B0BBF1000F09D141463C
:103FB0002046FFF7A1FF20B18BF311882846BDE80A
:103FC000F88FD4E90A12A7EB050B521A934528BFC4
:103FD0009346BBF1400F1BD9334601F1400251F823
:103FE000040B914243F8040BF9D1A36A40364035E3
:103FF0004033A362D4E90A239A4202D32046FFF752
:1040000095FF8AF31188BD42D8D289F31188C9E798
:1040100030465A46FCF748FFA36A5E445D445B4461
:10402000A362E7E710B5029C0433017203FB04218D
:10403000C460C0E906130023C0E90A33039B03638D
:10404000049BC0E90000C0E90422C0E908424363C0
:1040500010BD0000026A6FF00101C260426AC0E94F
:1040600004220022C0E90A22FEF7BEBBD0E90423E5
:104070009A4201D1C26822B9184650F8043B0B603D
:10408000704700231846FAE7C3680021C26901336C
:10409000C3604369134482699342436124BF436A06
:1040A0004361FEF795BB000038B504460D46E36852
:1040B0003BB1236900201A1DA262E2691344E36246
:1040C00007E0237A33B929462046FEF771FB002822
:1040D000EDDA38BD6FF00100FBE7000003691960FD
:1040E000C268013AC260C2691344826993420361A3
:1040F00024BF436A036100238362036B03B1184743
:104100007047000070B530230D460446114683F316
:104110001188866A2EB9FFF7C7FF10B186F31188A0
:1041200070BDA36A1D70A36AE26A01339342A36261
:1041300004D3E16920460439FFF7D0FF002080F363
:104140001188EDE72DE9F84F04460D469046994653
:104150004FF0300A8AF311880026B346A76A4FB998
:1041600049462046FFF7A0FF20B187F3118830466B
:10417000BDE8F88FD4E90A073A1AA8EB0607974278
:1041800028BF1746402F1BD905F1400355F8042BD3
:104190009D4240F8042BF9D1A36A40364033A36214
:1041A000D4E90A239A4204D3E16920460439FFF78F
:1041B00095FF8BF311884645D9D28AF31188CDE754
:1041C00029463A46FCF770FEA36A3D443E443B4410
:1041D000A362E5E7D0E904239A4217D1C3689BB1F3
:1041E000836A8BB1043B9B1A0ED01360C368013BFA
:1041F000C360C3691A4483699A42026124BF436A57
:104200000361002383620123184670470023FBE704
:1042100000F060BA014B586A704700BF000C0040C4
:10422000034B002258631A610222DA60704700BF14
:10423000000C0040014B0022DA607047000C004087
:10424000014B5863704700BF000C0040024B034A0B
:104250001A60034A5A6070474C5100207051002088
:1042600000000220074B494210B55C68201A084044
:104270001968821A8A4203D3A24201D85A6010BD3B
:104280000020FCE74C51002008B5302383F311884F
:10429000FFF7E8FF002383F3118808BD04480121DC
:1042A000044B03600023C0E901330C3000F016B961
:1042B0005451002089420008CB1D083A23F007031F
:1042C000591A521A012110B4D2080024C0E900433F
:1042D00084600C301C605A605DF8044B00F0FEB83E
:1042E0002DE9F84F364ECD1D0F46002818BF064663
:1042F000082A4FEAD50538BF082206F10C08341DFC
:104300009146404600F006F909F10701C9F1000E97
:10431000224624686CB9404600F006F93368CBB3F6
:1043200008224946E8009847044698B340E90267E6
:1043300030E004EB010CD4F804A00CEA0E0C0AF1F6
:104340000100ACF1080304EBC0009842E0D9A0EBF7
:104350000C0CB5EBEC0F4FEAEC0BD9D89C421CD2FD
:1043600004F10802AB45A3EB02024FEAE2026260ED
:1043700009D9691CED43206803EBC1025D44556017
:1043800043F8310022601C465F60404644F8086BE9
:1043900000F0CAF82046BDE8F88FAA45216802D18E
:1043A00011602346EFE7013504EBC50344F83510EF
:1043B00003F10801401AC01058601360F1E700BF14
:1043C00054510020F8B550F8043C044650F8085CFD
:1043D000A0F1080607332F1D0C35DB0840F8043C1C
:1043E000284600F097F83B469F421A6801D0B34236
:1043F00028D20AB1964225D244F8082C54F8042C4D
:104400001E60013254F8081C06EBC200814206D13E
:104410004868024444F8042C0A6844F8082C586898
:10442000411C03EBC1018E4207D154F8042C013228
:1044300002445A6054F8082C1A602846BDE8F84037
:1044400000F072B81346CFE7FEE7000070B51B4BD3
:104450000025044686B058600E4685620163FEF76B
:10446000EDFE04F11003A560E562C4E904334FF0EA
:10447000FF33C4E90044C4E90635FFF7CBFE2B4601
:10448000024604F134012046C4E9082380230C4A83
:104490002565FEF743F901230A4AE060009203759F
:1044A000684672680192B268CDE90223064BCDE9F5
:1044B0000435FEF75BF906B070BD00BF1034002074
:1044C000444E0008494E000849440008024AD36A95
:1044D0001843D062704700BFA8310020C0E9000037
:1044E000816070478368013B002B10B583600CDA54
:1044F000074BDC684368A061206063601C60446017
:104500000520FEF77DF8A06910BD0020FCE700BF84
:10451000A831002008B5302383F31188FFF7E2FFAC
:10452000002383F3118808BD08B5302383F3118875
:1045300083680133002B836007DC036800211A685D
:10454000026050601846FEF787F8002383F3118855
:1045500008BD00004B6843608B688360CB68C36014
:104560000B6943614B6903628B6943620B680360AB
:104570007047000008B53C4B40F2FF713B48D3F850
:1045800088200A43C3F88820D3F8882022F4FF62E9
:1045900022F00702C3F88820D3F88820D3F8E0205F
:1045A0000A43C3F8E020D3F808210A43C3F80821DE
:1045B0002F4AD3F808311146FFF7CCFF00F5806091
:1045C00002F11C01FFF7C6FF00F5806002F138011F
:1045D000FFF7C0FF00F5806002F15401FFF7BAFF5A
:1045E00000F5806002F17001FFF7B4FF00F5806014
:1045F00002F18C01FFF7AEFF00F5806002F1A80127
:10460000FFF7A8FF00F5806002F1C401FFF7A2FFE9
:1046100000F5806002F1E001FFF79CFF00F580608B
:1046200002F1FC01FFF796FF02F58C7100F5806046
:10463000FFF790FF00F01AF90E4BD3F8902242F0EA
:104640000102C3F89022D3F8942242F00102C3F889
:1046500094220522C3F898204FF06052C3F89C20A2
:10466000054AC3F8A02008BD0044025800000258C3
:10467000504E000800ED00E01F00080308B500F0F0
:10468000FDF9FEF725F8104BD3F8DC2042F040028C
:10469000C3F8DC20D3F8042122F04002C3F804213F
:1046A000D3F80431094B1A6842F008021A601A68FC
:1046B00042F004021A60FEF79BFDFEF703FDBDE821
:1046C0000840FEF77DBA00BF0044025800180248B7
:1046D00070470000114BD3F8E82042F00802C3F8FD
:1046E000E820D3F8102142F00802C3F810210C4A48
:1046F000D3F81031D36B43F00803D363C722094BBF
:104700009A624FF0FF32DA6200229A615A63DA60ED
:104710005A6001225A611A60704700BF0044025873
:104720000010005C000C0040094A08B51169D3680C
:104730000B40D9B29B076FEA0101116107D5302305
:1047400083F31188FDF7DEFF002383F3118808BD92
:10475000000C0040064BD3F8DC200243C3F8DC20F9
:10476000D3F804211043C3F80401D3F8043170478F
:104770000044025808B53C4B4FF0FF31D3F880207D
:1047800062F00042C3F88020D3F8802002F000429B
:10479000C3F88020D3F88020D3F88420C3F8841095
:1047A000D3F884200022C3F88420D3F88400D86F83
:1047B00040F0FF4040F4FF0040F4DF4040F07F0055
:1047C000D867D86F20F0FF4020F4FF0020F4DF40CE
:1047D00020F07F00D867D86FD3F888006FEA405088
:1047E0006FEA5050C3F88800D3F88800C0F30A007D
:1047F000C3F88800D3F88800D3F89000C3F890106D
:10480000D3F89000C3F89020D3F89000D3F8940028
:10481000C3F89410D3F89400C3F89420D3F894000C
:10482000D3F89800C3F89810D3F89800C3F89820EC
:10483000D3F89800D3F88C00C3F88C10D3F88C0010
:10484000C3F88C20D3F88C00D3F89C00C3F89C10DC
:10485000D3F89C10C3F89C20D3F89C30FCF706FEDC
:10486000BDE8084000F0F2B80044025808B5012243
:10487000534BC3F80821534BD3F8F42042F0020203
:10488000C3F8F420D3F81C2142F00202C3F81C2123
:104890000222D3F81C314C4BDA605A689104FCD5E3
:1048A0004A4A1A6001229A60494ADA6000221A6173
:1048B0004FF440429A61444B9A699204FCD51A68BD
:1048C00042F480721A603F4B1A6F12F4407F04D09A
:1048D0004FF480321A6700221A671A6842F0010208
:1048E0001A60384B1A685007FCD500221A611A6901
:1048F00012F03802FBD1012119604FF0804159605C
:104900005A67344ADA62344A1A611A6842F48032C9
:104910001A602C4B1A689103FCD51A6842F4805235
:104920001A601A689204FCD52C4A2D499A6200221A
:104930005A63196301F57C01DA6301F2E7119963A7
:104940005A64284A1A64284ADA621A6842F0A8525D
:104950001A601C4B1A6802F02852B2F1285FF9D194
:1049600048229A614FF48862DA6140221A621F4A33
:10497000DA641F4A1A651F4A5A651F4A9A6532232C
:104980001E4A1360136803F00F03022BFAD10D4A7D
:10499000136943F003031361136903F03803182B01
:1049A000FAD14FF00050FFF7D5FE4FF08040FFF7EF
:1049B000D1FE4FF00040BDE80840FFF7CBBE00BF7E
:1049C00000800051004402580048025800C000F026
:1049D000020000010000FF01008890082220400032
:1049E00063020901470E0508DD0BBF01200000200E
:1049F000000001100910E000000101100020005229
:104A000008B50348FCF704FFBDE80840FEF73EBCCC
:104A10006424002008B50348FCF7FAFEBDE808400E
:104A2000FEF734BCD024002008B50348FCF7F0FEA4
:104A3000BDE80840FEF72ABC3C25002008B5FFF77A
:104A400073FEBDE80840FEF721BC000008B509214F
:104A50007A20FCF763FF07213220FCF75FFF0C216F
:104A60002720FCF75BFF0C213520FCF757FF0C21BA
:104A70005220BDE80840FCF751BF000008B5FFF721
:104A800079FE00F00DF8FDF707F9FDF7DFFAFDF705
:104A9000B1F9FFF71DFEBDE80840FFF7B9BB000004
:104AA0007047000010B501390244904201D1002046
:104AB00005E0037811F8014FA34201D0181B10BD87
:104AC0000130F2E7034611F8012B03F8012B002A0D
:104AD000F9D1704765373165396264633261663197
:104AE000383530660000000012100000121100007E
:104AF0001213000053544D333248373F3F3F0053A9
:104B0000544D3332483733782F3732780053544D71
:104B10003332483734332F3735332F3735300000B1
:104B200001105A00031059000120580003205600BC
:104B300010000240080002400008024000000B0084
:104B400028000240080002400408024006010C0050
:104B500040000240080002400808024010020D0018
:104B600058000240080002400C08024016030E00E4
:104B7000700002400C0002401008024000040F00C8
:104B8000880002400C000240140802400605100094
:104B9000A00002400C00024018080240100611005C
:104BA000B80002400C0002401C08024016072F000B
:104BB00010040240080402402008024000083800A7
:104BC0002804024008040240240802400609390073
:104BD000400402400804024028080240100A3A003B
:104BE00058040240080402402C080240160B3B0007
:104BF000700402400C04024030080240000C3C00EB
:104C0000880402400C04024034080240060D4400AF
:104C1000A00402400C04024038080240100E450077
:104C2000B80402400C0402403C080240160F460043
:104C300000960000000000000000000000000000DE
:104C4000000000000000000000000000591C0008E7
:104C5000451C0008811C00086D1C0008791C000818
:104C6000651C0008511C00083D1C00088D1C000834
:104C700000000000711D00085D1D0008991D00085E
:104C8000851D0008911D00087D1D0008691D000894
:104C9000551D0008A51D00080000000001000000CF
:104CA0000000000063300000A44C00080032002027
:104CB000103400204172647550696C6F7400254295
:104CC0004F415244252D424C002553455249414CF9
:104CD000250000000200000000000000911F0008F5
:104CE0000120000840004000C04C0020D04C0020B3
:104CF00002000000000000000300000000000000AF
:104D0000492000080000000010000000E04C0020D6
:104D1000000000000100000000000000FC4F002027
:104D2000010102005D2B00086D2A0008092B000814
:104D3000ED2A0008430000003C4D00080902430032
:104D4000020100C032090400000102020100052432
:104D500000100105240100010424020205240600BC
:104D600001070582030800FF09040100020A000090
:104D70000007050102400000070581024000000015
:104D800012000000884D00081201100102000040CE
:104D90000912415700020102030100000403090443
:104DA00025424F415244250041524B56365800305F
:104DB0003132333435363738394142434445460081
:104DC000000000200000020002000000000000308F
:104DD000000004000800000000000024000008009B
:104DE000040000000004000000FC000002000000BD
:104DF00000000430008000000800000000000038BF
:104E0000000001000100000000000000A5210008D2
:104E10005D240008092500084000400034510020AE
:104E200034510020010000004451002080000000A7
:104E30004001000008000000000100000010000018
:104E4000080000006D61696E0069646C6500000017
:104E50000000802A00020000AAAAAAAA00000024DA
:104E6000FFFF00000000000000A00A00000000009A
:104E700000000000AAAAAAAA00000000FFFF00008C
:104E80000000000000000000000000020000000020
:104E9000AAAAAAAA00000001FFFF0000000000006B
:104EA0000000080020000A0000000000AAAAAAAA28
:104EB00010000500FFFF0000000800007700000060
:104EC0004014020028000000AAAAAAAA00000100BB
:104ED000FFFF0000000000000700000000200001AC
:104EE00000000000AAAAAAAA00100000FFFF00000C
:104EF000000000070000000000410000000000006A
:104F0000AAAAAAAA00400000FFFF000000000000BB
:104F1000000000000004004000000000AAAAAAAAA5
:104F200000040040FFFF000000000000000000003F
:104F30000001150000000000AAAAAAAA000115009D
:104F4000FFFF000000000000000000000000000063
:104F500000000000AAAAAAAA00000000FFFF0000AB
:104F60000000000000000000000000000000000041
:104F7000AAAAAAAA00000000FFFF0000000000008B
:104F800000000000000000003900000000000000E8
:104F900000001E0000000000FF0000001834002088
:104FA0003C250020D02400206424002000000000C4
:104FB000F44A000883040000FF4A0008500400007F
:104FC0000D4B00080096000000000800960000004D
:104FD00000080000040000009C4D000800000000D4
:104FE00000000000000000000000000000000000C1
:044FF00000000000BD
:00000001FF
